:020000040800F2
:10000000104000205D170008291700082B17000872
:100010002D1700082F1700083117000800000000F6
:10002000000000000000000000000000331700087E
:1000300035170008000000003717000839170008BE
:10004000891700088D1700089117000895170008F8
:10005000991700089D170008A1170008A5170008A8
:10006000A9170008AD170008B1170008B517000858
:10007000B9170008BD170008C1170008C517000808
:10008000C9170008CD170008D1170008D5170008B8
:10009000D9170008DD170008E1170008E517000868
:1000A000E9170008ED170008F1170008F517000818
:1000B000F9170008FD1700080118000805180008C6
:1000C000091800080D180008111800081518000874
:1000D000191800081D180008211800082518000824
:1000E000291800082D1800083118000835180008D4
:1000F000391800083D180008411800084518000884
:10010000491800084D180008511800085518000833
:10011000591800085D1800086118000865180008E3
:10012000691800086D180008711800087518000893
:100130007918000800000000000000000000000026
:100140000000000000000000000000007D18000812
:100150008118000885180008891800088D18000803
:100160009118000895180008991800089D180008B3
:10017000A1180008A518000800000000A918000830
:10018000AD180008B1180008B5180008B918000823
:10019000BD180008C118000800000000C5180008BC
:1001A000000000000000000000000000C918000866
:1001B000CD180008D1180008000000000000000061
:1001C000000000000000000000000000000000002F
:1001D000000000000000000000000000D51800082A
:1001E00070B582B0054600F099FA06460DB90120B7
:1001F00076BD05F140042078012801D1022076BDAA
:1002000001202070607830B92070284600F085FA0F
:1002100041F28830A060286833460168AA6821F45A
:10022000F851521E41EA022100220160A0680090AC
:100230002021284600F0C1F9010022D12968124B83
:100240000A681A406B6842EA0362EB681A43EB697A
:100250001A432B6A1A430D4B0A6029684A681A40F0
:100260002B6942EA03426B691A43AB691A434A603D
:1002700029680A6842F001020A60002161600121D8
:1002800061700021217076BD2FFFFF00FEF8E0FFB6
:1002900010B508B9012010BD00F1400421780129F2
:1002A00001D1022010BD0121217001680A685208A5
:1002B00052000A6000F038FA002060606070207020
:1002C00010BD2DE9F84304460D46164604F14007DB
:1002D00000F024FA80463878012808BF022024D094
:1002E00001203870787801281AD1002043467860C0
:1002F000022078700022009600F020F9814688B92B
:1003000000F015F8686A40B90096434600F0FEF820
:10031000814638B921680220C8600120787001E068
:100320004FF00209002038704846BDE8F2830022F1
:100330002946204664E12DE9F843044604F14006CD
:100340000F46154600F0EAF9804620683178012909
:1003500000F1200908BF022034D000F035F82ED17A
:100360000021716047B3122171700169491CE1627B
:100370000169491CA1626762416921F040614161E4
:100380000EE00122042100F0C3F8010011D1606ADF
:10039000411C6162007889F80000E06A401EE0625A
:1003A000E06A009543460028EBD100F0AFF800F07A
:1003B00066F80121717003E000F05BF800E00220B4
:1003C00000213170BDE8F28301213170717801297B
:1003D00070472DE9F84304460F46154604F14006E0
:1003E00000F09CF98046206881693278012A00F18A
:1003F000200908BF02203AD0012232707278012A07
:1004000032D10022726067B3222272700269521CDC
:10041000A2630269521C62632763426922F0406250
:1004200042F080624261206881610EE00122062173
:1004300000F06EF8010011D1206B411C216399F886
:1004400000100170A06B401EA063A06B0095434696
:100450000028EBD100F05AF800F011F8012171707A
:1004600003E000F006F800E0022000213170BDE852
:10047000F283706840F0080070600120704701004E
:1004800002D122680221D16070472DE9F843044669
:10049000894616461F4600F041F9804604F14005A2
:1004A0002878012808BF02202ED001202870687803
:1004B000012826D10020434668604220687000224F
:1004C000009700F03BF801001CD100F023F841F444
:1004D00080010160F068C9F828004FF000624946C9
:1004E000204600F08DF8009743460122082100F0D5
:1004F0000FF8010006D122680821D160012169703E
:1005000000E0022000212970BDE8F28301220221CF
:10051000204652E02168306888622168706848622D
:100520002168B068C86220680168326921F440011E
:10053000114370477170B16800910022202120465C
:100540003BE02DE9F04182B004468846174600F0B2
:10055000E5F804F140063178012908BF02202AD0CD
:10056000FFF732FF23D10021034671608221FFF79C
:10057000E1FF0546E0B9206801687A6821F00801CA
:1005800011430160786808280AD121683868086337
:1005900021681020C8602068016841F48011016062
:1005A0004FF040624146204600F02AF800E0022564
:1005B000002030702846BDE8F6812DE9F041044660
:1005C0000D4690461F46069E20688068284018BF4A
:1005D0000120404511D016F1010FF5D026B100F0F1
:1005E0009DF8C01B8642EFD2042084F84100606C65
:1005F00040F001006064012000E00020BDE8F081CF
:10060000F0B54B6A002B18BFB2F1406F03D08B6A74
:1006100004685B1E23618C69002C2BD00D6A036873
:100620007DB100F066F80F6800F069F836B1D1F8D6
:100630000CC04CEA040434432C4315E045EA0400A2
:1006400016E0CE6A0F6B4D6A3E434F6B3E430F6818
:1006500035434E6945EA8646CD693DB1D1F80CC0B7
:100660004CEA060635432C433C430FE044EA0600BF
:10067000384313E00B6AA3B1036800F03AF800F0C6
:100680003EF84EB1CF683C4334432C431443B2F19F
:10069000406F5C611AD1F0BD45EA04001043586117
:1006A000F0BDCD69B5B1CB6A0C6B23434C6B2343D2
:1006B0004C6A23434C6943EA8443CC6823432B436D
:1006C00004681343B2F1406F636111D00068496858
:1006D0008161F0BD4D6A5DB1CB6A0C6B006823434C
:1006E0004C6B496923432B4343EA814111434161E8
:1006F000F0BD8C68DC61CC6A0D6BCE6970472C4311
:100700004D6B2C434D6A2C434D6944EA85440D6979
:100710002C430D6A2C438D6970477047014840682F
:10072000704700BF00000020704700002DE9F04135
:10073000040082B04FF0000817D02078DFF80C5486
:10074000C00747D5A86800F00C00042807D0A868A7
:1007500000F00C0008280AD16868400207D5286814
:10076000800337D56068002834D1012040E16068FB
:10077000B0F5803F09D008B928680AE0B0F5A02F8D
:10078000286806D140F480202860286840F4803032
:1007900005E020F480302860286820F4802028605C
:1007A000606858B1FFF7BAFF07462868800311D484
:1007B000FFF7B4FFC01B6528F7D316E1FFF7AEFFC4
:1007C00007462868800305D5FFF7A8FFC01B6528EA
:1007D000F7D30AE12078800718D5A86810F00C0F2D
:1007E00007D0A86800F00C00082825D168684002EE
:1007F00022D42868800702D5E0680128B5D128688E
:10080000216920F0F80040EAC10028602078000744
:1008100043D560690028686F30D040F001006867F8
:10082000FFF77CFF0746686F800736D4FFF776FF37
:10083000C01B0328F7D3D8E0E068002828680ED052
:1008400040F001002860FFF769FF0746286880072D
:10085000D5D4FFF763FFC01B0328F7D3C5E04008DA
:1008600040002860FFF75AFF074628688007CDD56B
:10087000FFF754FFC01B0328F7D3B6E04008400041
:100880006867FFF74BFF0746686F800705D5FFF7DE
:1008900045FFC01B0328F7D3A7E0207840075CD5AD
:1008A000286CC0000AD4286C4FF0010840F080503A
:1008B0002864286C00F0805000900098DFF898625F
:1008C0003068C0050FD4306840F480703060FFF7A6
:1008D00025FF07463068C00505D4FFF71FFFC01B82
:1008E0006528F7D381E0A068012808D008B9286FEF
:1008F00009E00528286F06D140F004002867286F1A
:1009000040F0010005E0400840002867286F20F013
:1009100004002867A06841F2893658B1FFF7FEFE4F
:100920000746286F800711D4FFF7F8FEC01BB042BE
:10093000F7D35AE0FFF7F2FE0746286F800705D588
:10094000FFF7ECFEC01BB042F7D34EE0B8F1000F4A
:1009500003D0286C20F080502864A069002846D07D
:10096000A96801F00C0108293FF4FFAE02282868AD
:1009700020F0807028602DD1FFF7D0FE0746286850
:10098000800105D5FFF7CAFEC01B0328F7D32CE072
:10099000E069216A0843616A40EA8110A16A891E00
:1009A000C903090C40EA0140E16A40EA016040F0F5
:1009B00000506860286840F080702860FFF7AEFE45
:1009C00007462868800112D4FFF7A8FEC01B032841
:1009D000F7D30AE0FFF7A2FE07462868800106D594
:1009E000FFF79CFEC01B0328F7D3032000E0002084
:1009F000BDE8F6812DE9F0410400884650D0574EFD
:100A0000306800F00F00404502D200F06EF847D188
:100A100020684E4F810712D5400703D5B86840F4CF
:100A2000E050B8602078000703D5B86840F4604013
:100A3000B860B868A16820F0F0000843B86020787A
:100A4000C00725D56068012802D13968890303E011
:100A50000228396802D1890102D421E089071FD513
:100A6000B968890840EA8100B860FFF757FE05467B
:100A7000B868616800F00C00B0EB810F08D0FFF798
:100A80004DFE401B41F289318842F1D303202AE018
:100A9000306800F00F00804504D200F026F801D045
:100AA000012020E02078400705D5B868E16820F4EF
:100AB000E0500843B8602078000706D5B86821697F
:100AC00020F4604040EAC100B86000F018F8BA684D
:100AD0002349C2F30312895CC8401D4908600F20F6
:100AE00000F044F80020BDE8F0813068000948EAD1
:100AF00000103060306800F00F004045704710B5BE
:100B0000184C606800F00C00042802D0082802D0BD
:100B100019E0154810BD2068002300F03F0220684E
:100B200040022068C0F388104CBF0F490949A1FB5F
:100B3000000100F03BF82168C1F30141491C490064
:100B4000B0FBF1F010BD034810BD000000380240BA
:100B50000C0000200024F40000700040003C024023
:100B60004C1700080438024040787D0138B50D4D1F
:100B7000044629784FF47A70B0FBF1F00A4909680D
:100B8000B1FBF0F000F0C1F850B9102C08D20022EF
:100B900021464FF0FF3000F09BF8AC60002032BDE2
:100BA000012032BD000000200C0000201B4213D1A8
:100BB000094236D12AB18446B0FBF2F002FB10C2E2
:100BC000704700F0C1B8FCD30022002370470B002F
:100BD0000200002100207047904271EB030CF6D315
:100BE00070B5B1FA81F4B3FA83F52C1BA340C4F1BC
:100BF000200532FA05F63343A2405FF00046E64096
:100C000002E05B085FEA3202841A71EB030524BF3D
:100C1000204629467641F4D302000B003000002123
:100C200070BD012ACFD970B5140C20D0B1FA81F46F
:100C3000B2FA82F5C4F120046419B4F12006D6D3C7
:100C4000B2405FF00044F440002502E052085FEA41
:100C50003303C61A71EB020E24BF3046714664415D
:100C60006D41F3D302000B002000290070BD0C463B
:100C7000B1FBF2F102FB11452D0445EA1045B5FB2D
:100C8000F2F402FB145580B240EA0545B5FBF2F0E0
:100C900002FB105240EA044070BD00000901002828
:100CA00002D4244A11547047234A00F00F00104424
:100CB00000F8041C704721494FF6FF030A68000240
:100CC00000F4E0601A4010431D4A1043086070476A
:100CD00038B51A4B1B68C3F30223C3F10704052C74
:100CE00028BF04241D1D072D34BF0023DB1E012552
:100CF00005FA04F4641E2140994005FA03F35B1ED3
:100D00001A401143BDE83440C8E7401EB0F1807F6F
:100D100010B501D3012010BD0A4C0F2160604FF0C7
:100D2000FF30FFF7BBFF0020A060072020600020FD
:100D300010BD000000E400E018ED00E00CED00E064
:100D40000000FA0510E000E070470000DFF87803CB
:100D50002DE9F041DFF8744384B020602046FFF7AE
:100D600097FA002829D100F0B5F9DFF86453002084
:100D7000E8614FF44076286268626861E86228633F
:100D800068634FF44050E8600020A8640120686464
:100D9000102028644FF48000E86401206060102077
:100DA000A060E060192020610020A061E061206265
:100DB00020466661FFF714FA00287AD1204600F039
:100DC00080F8002875D14FF4807041F28838A8610E
:100DD000352000F033F900286BD14020AE61A863C4
:100DE0004120E863052028604FF040776F6243465A
:100DF00005F1380200F061F800285AD1B720AE6141
:100E0000286000206862204600F020F9002850D1B8
:100E100000F017F900284CD14146204600F03CF97B
:100E2000002846D1204600F0BCF8002841D1AE6130
:100E300005206F62424628600120A86200F002F996
:100E4000002836D100F0F5F8002832D115204246AE
:100E500028600120A86200F0F5F8002829D1424658
:100E60000DF1010100F0E7F818BB204600F0EEF8A4
:100E7000F8B900F0D2F84246204601F0F80141F0FE
:100E8000060100F0D1F8A0B900F086F888B9EC208E
:100E9000AE6128604FF44060E8610A206F6201AAE9
:100EA000686100200290294601902046FFF749FB27
:100EB00000B1012004B0BDE8F08129462046FFF7CB
:100EC000E4BA2DE9F0410446814D4FF4407041F2FF
:100ED0008838A861662028600020686282B000F02F
:100EE000B0F8002850D199204246286000F0AAF8B6
:100EF000002849D166204FF4807728604246AF61D0
:100F000000F0A0F800283FD199204246286000F068
:100F100099F8002838D14FF47A7000F055F941461D
:100F2000204600F0B9F800282ED10520AF612860D6
:100F30004FF080766E620120A86200F082F80028EF
:100F400022D100F076F8F8B90620AF6100F076F80B
:100F5000D0B90220434600F090F829466E62FFF7B0
:100F6000ADFF88B90120AF6128604246A8629DF8B4
:100F70000000294640F040008DF8000000F063F8C2
:100F800010B900F009F808B1012003E0282000F0B2
:100F90001BF90020BDE8F681424669462046FFF76E
:100FA000CAB970B500F070F84FF040706862012067
:100FB000A8620520286082B0324600F043F800287D
:100FC00024D1324600F036F800BB152032462860A6
:100FD0000120A86200F036F8C0B932460DF10101D7
:100FE00000F029F890B9204600F030F870B900F010
:100FF00014F83246204641F0C00100F015F828B937
:10100000324669462046FFF796F908B1012076BDC1
:10101000282000F0D9F8002076BD9DF801100120AD
:1010200028600220A86270478DF801102946FFF75A
:1010300048B9424669462046FFF7CBB928600020F0
:101040006862424629462046FFF73BB970B500F07A
:101050001BF806202860002068623246FFF7F2FF86
:1010600048B90220334600F008F84FF0407068623B
:10107000FFF723FF00B1012070BDA86305F138021E
:10108000E8630520286070470446114D4FF4407016
:1010900041F28836A861704710B50D4C4FF440728C
:1010A000A261052222604FF0407262620022A263B8
:1010B0000122E2630B4604F138022146FFF7E5F90D
:1010C00000B1012010BD0000001000A06040002011
:1010D0001040002010B586B03448016A344C41F00D
:1010E00002010162016A01F00201009100990168A8
:1010F00041F002010160016821F002010160816993
:1011000041F002018161816901F0020100910099C1
:10111000816941F004018161816901F0040100915C
:101120000099816941F010018161816901F010012C
:1011300000910099816941F008018161806901A9EC
:1011400000F0080000900098402001900A200590CF
:1011500002200290012003900220049000F030F859
:10116000042001A90190092005900020039000F0BF
:1011700027F84FF400700F4C019001A900F020F8FF
:101180004FF4806001A9019000F01AF8042001A931
:101190000190094800F02CF84FF4005001A901908B
:1011A000064800F025F806B010BD000018380240CF
:1011B000000402400008024000100240000C0240FF
:1011C000204600F015B8000038B50446FFF7A6FA2F
:1011D00014F1010F054602D0044800782418FFF7E7
:1011E0009DFA401BA042FAD331BD00BF0000002091
:1011F0002DE9F84F02460023DFF89481DFF894913F
:10120000DFF894A14FF00F0B0C680120984000EA22
:10121000040E864540F0B6804D689C00022D18BF34
:10122000122D0FD1DD0802EB850C04F01C050BFA22
:1012300005F7DCF82060BE430F6907FA05F5354372
:10124000CCF8205016680F794FEA430C032505FAB5
:101250000CF5ED432E4007F0030707FA0CF73E4369
:1012600016604E68012E18BF022E03D0112E18BF33
:10127000122E0FD19668CF682E4007FA0CF73E4326
:101280009660566826EA00004E68C6F300169E4037
:1012900030435060D06828408D6805FA0CF528432B
:1012A000D0604868C0006DD5DAF8000004F00C0684
:1012B0000BFA06F440F48040CAF80000DAF80000A7
:1012C00000F4804000900098980859F8205025EAD2
:1012D0000404324DAA4208BF002522D0304DAA4254
:1012E00008BF01251DD02F4DAA4208BF022518D0E6
:1012F0002D4DAA4208BF032513D02C4DAA4208BF8A
:1013000004250ED02A4DAA4208BF052509D0294D33
:10131000AA4208BF062504D0274DAA420CBF0725C4
:101320000825B5402C4349F82040D8F800406FEA22
:101330000E0000EA040C4C68E40348BF4EEA0C0CB3
:10134000C8F800C0D8F8044000EA040C4C68A403B4
:1013500048BF4EEA0C0CC8F804C0D8F8084000EAB0
:10136000040C4C68E40248BF4EEA0C0CC8F808C0F4
:10137000D8F80C4020404C68A40248BF4EEA000058
:10138000C8F80C005B1C102BFFF43EAFBDE8F18FDA
:10139000003C01400838014044380240000002404F
:1013A0000004024000080240000C0240001002400D
:1013B0000014024000180240001C024070B592B0B8
:1013C00000F098F8474C00F0A0F8474D286840F42A
:1013D0000030286000F093F82867BFF34F8FE86E65
:1013E00043F6E076C0F34E31C0F3C90206EA41137A
:1013F00043EA8273236113465A1E002BF6D10A4634
:10140000511E002AF0D1BFF34F8F286840F480307E
:10141000286000F06FF800F07FF8012005904FF48D
:101420008030069002200B904FF480000C90192021
:101430000D904FF4C8700E9002200F90082010906D
:1014400005A8FFF773F900B1FEE700F079F800B1E5
:10145000FEE70F200621009002200190002002905C
:101460004FF4A05003904FF4805004906846FFF76B
:10147000C1FA00B1FEE7FFF769FC00B1FEE700F03A
:1014800039F8286820F40030286000F03EF828671A
:10149000BFF34F8F286820F480302860BFF34F8F50
:1014A000E86EC0F34E31C0F3C90206EA411343EAC5
:1014B0008273636213465A1E002BF6D10A46511EF0
:1014C000002AF0D100F01BF8084908604FF01040E6
:1014D000074942680A60006880F308881046804720
:1014E000FEE7000050EF00E014ED00E010E000E047
:1014F000AC400020BFF34F8FBFF36F8F7047BFF337
:101500004F8FBFF36F8F0020704700202060BFF324
:101510004F8FBFF36F8F704780B50748016841F464
:10152000807101600320FFF7C6FB0F20FFF71EFB51
:1015300000F004F8002002BD003C024070470000AB
:1015400070B582B000F020F840F4803000F030F840
:1015500006466068C00305D4FFF7E0F8801BA84288
:10156000F7D30DE0206840F4003000F021F8064683
:101570006068800306D4FFF7D1F8801BA842F7D338
:10158000032076BD002076BD08480168064C40F275
:10159000E93541F080510160006800F08050009012
:1015A00000982068704700000070004040380240FA
:1015B0002060FFF7B3B800000E480F4A016841F4FD
:1015C000700101600D48016841F0010101600021D6
:1015D000816001681140016009494160016821F49E
:1015E000802101600021C1604FF000600549086062
:1015F0007047000088ED00E0FFFFF6FE0038024073
:101600001030002408ED00E019E050F8041BCB076F
:1016100044BFA9F101035918121F0023042A41F8FD
:10162000043BF9D25FEA827C0B4604D54FF0000CF4
:10163000A1F800C09B1CD10744BF0021197050F8CD
:10164000042B002AE1D1704710B450F8041B79B183
:101650000268436802440830DC0744BFA9F1010472
:10166000E31852F8044B43F8044B091FF9D1ECE797
:1016700010BC704710B5074979441831064C7C44BA
:10168000163404E00A68081D114488470146A14247
:10169000F8D110BD2C0000004C0000004EF688511F
:1016A000CEF20001086840F470000860BFF34F8F6D
:1016B000BFF36F8F4FF00070E1EE100A704700002B
:1016C00049FFFFFFA00000001040002000000000C4
:1016D00079FFFFFF100000009400000000000020D0
:1016E0000000000000F00BF8002801D0FFF7C2FF57
:1016F0000020AFF30080FFF761FE00F002F8012048
:10170000704700F001B800000746384600F002F8C4
:10171000FBE7000080B5AFF30080024A11001820FB
:10172000ABBEFBE7260002007047FEE7FEE7FEE7E0
:10173000FEE770477047704700F000B80248416804
:101740000278891841607047000000200000000006
:101750000000000001020304060708090148804751
:1017600001480047B91500087D1700080100000076
:1017700000000000100000000024F400AFF300801F
:10178000FFF78CFFFFF7AEFFFFF7FEBFFFF7FEBFCF
:10179000FFF7FEBFFFF7FEBFFFF7FEBFFFF7FEBF7D
:1017A000FFF7FEBFFFF7FEBFFFF7FEBFFFF7FEBF6D
:1017B000FFF7FEBFFFF7FEBFFFF7FEBFFFF7FEBF5D
:1017C000FFF7FEBFFFF7FEBFFFF7FEBFFFF7FEBF4D
:1017D000FFF7FEBFFFF7FEBFFFF7FEBFFFF7FEBF3D
:1017E000FFF7FEBFFFF7FEBFFFF7FEBFFFF7FEBF2D
:1017F000FFF7FEBFFFF7FEBFFFF7FEBFFFF7FEBF1D
:10180000FFF7FEBFFFF7FEBFFFF7FEBFFFF7FEBF0C
:10181000FFF7FEBFFFF7FEBFFFF7FEBFFFF7FEBFFC
:10182000FFF7FEBFFFF7FEBFFFF7FEBFFFF7FEBFEC
:10183000FFF7FEBFFFF7FEBFFFF7FEBFFFF7FEBFDC
:10184000FFF7FEBFFFF7FEBFFFF7FEBFFFF7FEBFCC
:10185000FFF7FEBFFFF7FEBFFFF7FEBFFFF7FEBFBC
:10186000FFF7FEBFFFF7FEBFFFF7FEBFFFF7FEBFAC
:10187000FFF7FEBFFFF7FEBFFFF7FEBFFFF7FEBF9C
:10188000FFF7FEBFFFF7FEBFFFF7FEBFFFF7FEBF8C
:10189000FFF7FEBFFFF7FEBFFFF7FEBFFFF7FEBF7C
:1018A000FFF7FEBFFFF7FEBFFFF7FEBFFFF7FEBF6C
:1018B000FFF7FEBFFFF7FEBFFFF7FEBFFFF7FEBF5C
:1018C000FFF7FEBFFFF7FEBFFFF7FEBFFFF7FEBF4C
:0818D000FFF7FEBFFFF7FEBFAA
:040000050800177D5B
:00000001FF
